:100000000C94C5030C94E2030C94FD030C94E203DE
:100010000C94E2030C94E2030C94E2030C946A1D2A
:100020000C94E2030C948E1D0C94A1220C94E20318
:100030000C94E2030C94E2030C94E2030C94E203AC
:100040000C94E2030C94E2030C94E2030C94E2039C
:100050000C94E20380078007AC07AC0714083F0943
:100060003F093F093208CB08DC08DC082F68040090
:100070000351000001512C000000000000000000AE
:1000800000000251000000000000D85C1D001B00B1
:100090000600190005000000000000000000380004
:1000A000000000000000000034610400160007009A
:1000B00009000A0000000000000000003300287161
:1000C000000000000000296114001A00080015005B
:1000D00017000000000000000000130000000000F6
:1000E000000000002B0000000000000000000000E5
:1000F0000000000000000000000000000000000000
:100100002A00000000001C000B0011002C0004510C
:100110003078140035710000000018000D00100048
:100120000000000012000F0037000000D95C000042
:1001300000000000000000000C000E00360001006E
:1001400001000100000001000100000000000000AB
:1001500000000000620000000000000001003A0002
:100160003B003C003D00C05C0000000000000000BF
:100170005600000000000000000001003E003F00AB
:1001800040004100CB5C0000000000000000550072
:100190000100000000000000010042004300440094
:1001A0004500C35C00000000000000005400000097
:1001B000000000000000010000000000000000003E
:1001C000000000000000000000000000000000002F
:1001D0000000010000000000C45CCA5CBF5C0100BC
:1001E0006300570058004E00000000005F005C00F4
:1001F00059000000000061005E005B0000004B0041
:100200000000000000000000000060005D005A00D7
:1002100001000100010000000100010000000000D9
:1002200000000000000001000000000000000100CC
:1002300001000100010001000100000000000000B9
:1002400000000100000000000000000001001E008E
:100250001F0020002100220000000000000000001C
:1002600027002D0000000000000035000100010003
:10027000010001000100000000000000000030004B
:10028000000000000000000001000000000000006D
:10029000000000000000000000000000000000005E
:1002A00000000000640000000000010023000100C5
:1002B00001004A004B004E004D00000000003400D9
:1002C00024000100000000002F00260001000000B3
:1002D0000100000000000000000000002E002500CA
:1002E0000100010001000100000001000100000008
:1002F00000000000000000000100000000000000FD
:10030000010001007B00010001000100000000006D
:1003100000000000010000000000000000000100DB
:10032000010001004E00010001000000000000007B
:1003300000000100010000000000000001000100B9
:1003400001000100010001000000000000000000A9
:100350007D0000000000000000000100000000001F
:10036000000000000000000000000000000000008D
:100370000000000000004C00000000007C00500065
:100380000100010001000100010001000000000067
:100390004B00510001000000000001004F0001006F
:1003A000000001000000000000000000000001004B
:1003B00052000100010001000100000001000100E5
:1003C000000000000000000000000100000000002C
:1003D000000039000100AE00BC00BB0001000000BD
:1003E000000000000000010000000000000000000C
:1003F00001004900A800AA00A900010000000000B7
:1004000000000000010001000000000000004600A4
:1004100001000100010001000100000000000000D7
:1004200000000100000000000000000001000000CA
:1004300000000000000000000000000000000000BC
:1004400000000000000000000100000000000100AA
:10045000EF000100010001000100010001000000A7
:100460000000FD00EE00010000000000FF00F000B1
:10047000F200000001000000000000000000000089
:10048000FE00ED00F10000047F3F1F64321464326F
:1004900014783C1E1E140A052223252628292A2CFE
:1004A0002D2F3032333536383A3B3D3E40424345BE
:1004B00047494A4C4E5051535557595A5C5E6062F9
:1004C000646668696B6D6F71737577797B7D7F8109
:1004D000838587898A8C8E90929496989A9C9E9F09
:1004E000A1A3A5A7A8AAACAEAFB1B3B4B6B8B9BB27
:1004F000BCBEBFC1C2C3C5C6C7C9CACBCCCDCED096
:10050000D1D2D2D3D4D5D6D7D7D8D9D9DADADBDB82
:10051000DBDCDCDCDCDCDDDDDDDDDCDCDCDCDCDB19
:10052000DBDBDADAD9D9D8D7D7D6D5D4D3D2D2D162
:10053000D0CECDCCCBCAC9C7C6C5C3C2C1BFBEBC55
:10054000BBB9B8B6B4B3B1AFAEACAAA8A7A5A3A1C6
:100550009F9E9C9A98969492908E8C8A8987858388
:10056000817F7D7B79777573716F6D6B6968666468
:1005700062605E5C5A5957555351504E4C4A494738
:10058000454342403E3D3B3A3836353332302F2DDD
:100590002C2A292826252322FFAA7F554000010165
:1005A0000101010101010102020202020202020232
:1005B0000303030303030303040404040404040502
:1005C00005050505060606060607070707070808C6
:1005D0000808090909090A0A0A0B0B0B0C0C0C0D77
:1005E0000D0D0E0E0E0F0F0F101011111112121310
:1005F000131414151516161717181819191A1A1B8B
:100600001B1C1D1D1E1E1F202021222223242425E9
:100610002626272829292A2B2C2D2D2E2F30313222
:1006200032333435363738393A3B3C3D3E3F404132
:1006300042434445464748494A4C4D4E4F5051531A
:1006400054555658595A5B5D5E5F616264656668D1
:10065000696B6C6D6F7072737577787A7B7D7E8055
:1006600082838587888A8C8E8F91939596989A9CA1
:100670009EA0A2A3A5A7A9ABADAFB1B3B5B7BABCB5
:10068000BEC0C2C4C6C9CBCDCFD1D4D6D8DBDDDF86
:10069000E2E4E7E9EBEEF0F3F5F8FAFDFF09023BDF
:1006A00000020100A0FA0904000001030101000991
:1006B0002101010001224000070581030800010912
:1006C00004010001030000000921010100012232A0
:1006D0000007058303080001120110010000000853
:1006E000A0202D420100010200010A034D00540028
:1006F0003400300000001C03540068006F006D00DF
:1007000061007300440065006800610065007A00C4
:10071000650000000403090405010980A1018503A7
:1007200019012AB700150126B7009501751081003F
:10073000C0050C0901A101850419012AA0021501B7
:1007400026A002950175108100C005010906A101CE
:10075000050719E029E715002501950875018102B3
:100760009501750881030507190029FF150026FF6B
:10077000009506750881000508190129059505757C
:10078000019102950175039103C011241FBECFE5AD
:10079000D8E0DEBFCDBF11E0A0E6B0E0EAEDFDE4B9
:1007A00002C005900D92A232B107D9F723E0A2E270
:1007B000B1E001C01D92A532B207E1F70E943815E1
:1007C0000C94EB260C940000A82FB92F80E090E049
:1007D00041E050EA609530E009C02D91822797955D
:1007E000879510F084279527305EC8F36F5FA8F3D4
:1007F0000895EADF8D939D930895CF93CFB7CF935C
:10080000C395839BE9F7839B0EC0839B0CC0839B9E
:100810000AC0839B08C0839B06C0C091FC02C3959D
:10082000C093FC02A6C0DF93C091FB02DD27CD5F21
:10083000DC4F839B02C0DF91E6CF2F930F931F9372
:1008400000B32FEF03FB20F94F933F9310B34FEF0B
:10085000012703FB21F93BE031C04E7F012F10B38C
:10086000216028C0102F4D7F2260000000B329C0F6
:100870004B7F2460012F000010B32BC010B3477FC3
:1008800028602AC04F7E00B320612CC04F7D10B37A
:1008900020622FC04F7B00B3206432C0422700B3D8
:1008A00049934FEF0000102713FB20F910B31C7081
:1008B000C9F1297F91F2012703FB21F900B3237FBE
:1008C00089F2315058F1102713FB22F910B3277E1B
:1008D00079F2012703FB23F92F7C81F200B3102763
:1008E00013FB24F92F7971F200C010B3012703FB29
:1008F00025F92F7359F200C000B3102713FB26F916
:10090000223040F200C010B3012703FB27F9243046
:1009100028F64F77206810B30000F9CF10E81ABF0F
:1009200000271CC03B503195C31BD04010E81ABFB4
:100930000881033C11F10B3401F12091F802198177
:10094000110F1213EDCF4A81441F093669F10D32A0
:1009500011F0013E29F74F7009F0042F00930103B5
:100960003F914F911F910F912F91DF91CAB7C7FD12
:1009700047CFCF91CFBFCF9118952091010322236C
:1009800079F31091FF02112309F044C034300AF4C6
:1009900043C03093FF022093FA021091FB023BE028
:1009A000311B3093FB0238C00091FF02013094F5F7
:1009B0000AE54F7049F43091840034FD2FC0009354
:1009C0008400C5EDD2E02EC0433059F0443091F0A0
:1009D0003091E00234FD22C00093E002C1EED2E08B
:1009E00021C03091190334FD19C000931903CAE1E5
:1009F000D3E018C03091EC0234FD10C00093EC023B
:100A0000CDEED2E00FC02795A8F45150A9F4220FE3
:100A10000000F9CF4AE503C042ED01C0432FC4E115
:100A2000D0E032E011B31C60939A11BB02B320E412
:100A30001CE05F93012756E002BB279520F451503C
:100A400021F4220FF9CF012756E000003B5A02BBE8
:100A5000D0F2279528F4515029F4220F0000F9CF45
:100A6000012756E0279502BB20F4515021F4220FB4
:100A7000F9CF012756E02991332302BB21F6037FEA
:100A800010910003110FC651D04002BB11F010931A
:100A9000F80210E81ABF086011B3137F402F437F9C
:100AA0005F9100C000C002BB11BB42BB59CF81E0C7
:100AB000089581E008950C94590508950C945D05FE
:100AC0001F93CF93DF9300D000D01F92CDB7DEB736
:100AD00049835A836B833091250189819A81311131
:100AE00014C0662359F0222349F00E94780B182F76
:100AF000682F89819A810E94210B03C00E944C0BB0
:100B0000182F69817A81812F04C00E94780B698136
:100B10007A810F900F900F900F900F90DF91CF91EF
:100B20001F910C94A612FC01262F408151816281F5
:100B3000738184810C94600581E00895CF93DF93E5
:100B4000EC0160E00E949305BE01DF91CF910C940F
:100B50005E050C94EF130C94EB1308950E94CB09DF
:100B60000E94AD052FEB87E299E021508040904034
:100B7000E1F700C000000C94C7220F931F93CF939E
:100B8000DF938C0161E00E949305EC01B8010E94A3
:100B90005B05882309F44BC0B801CE010E94331DC8
:100BA000882309F444C0B801CE010E948320882321
:100BB000F1F1B801CE010E94971E8823C1F1B8015E
:100BC000CE010E94DF1F882391F1B801CE010E945F
:100BD000771B882361F1F8018281882309F1CB35E5
:100BE0008DE5D807C1F050F4C115FCE5DF0781F0B1
:100BF000CF3DDC45A9F40E94AF1019C0CC35EDE51E
:100C0000DE0761F0CD35DD4559F40E94F20F08C0D2
:100C10000E94AE050CC00E94FB0F02C00E94FE0F96
:100C2000C801DF91CF911F910F910C94570580E07F
:100C3000DF91CF911F910F9108950E944B2280E088
:100C40000E94BF1D0C943B060E94571C0E943E064A
:100C50000C94512208950C942A0681E008950C9476
:100C60002D060895CF93C82F0E942B068C2F0E942B
:100C70002F06CF91089580E00C9432060E94B8218F
:100C80000C9432060E94B82190912401891721F01A
:100C9000809324010C9432060895CF93DF93CDB74F
:100CA000DEB72B970FB6F894DEBF0FBECDBF4F83D4
:100CB000588769877A878B8761110E943E0F9E0152
:100CC0002F5F3F4F86E0F90111928A95E9F785E0A1
:100CD000FE013796D90101900D928A95E1F789813D
:100CE0009A814C815D81452B31F09F3F31F491E039
:100CF0008F3F19F403C091E001C090E090FF09C05C
:100D000049815A816B817C818D819E810E945F0E19
:100D100005C0C9010E949C058111F2CF2B960FB628
:100D2000F894DEBF0FBECDBFDF91CF910895FC01D7
:100D3000808191810E94BA0B0895CF93882309F492
:100D400048C0C82F8CEF8C0F813AD0F46C2F809163
:100D50006200909163000E940722882349F06C2F63
:100D600080916200909163000E943F220E94600F78
:100D70006C2F80916200909163000E943D220CC014
:100D800080E28C0F883058F4C77081E001C0880F72
:100D9000CA95EAF70E94210FCF910C94600FEBE502
:100DA000EC0FE33040F4F0E0ED54FF4F808190E031
:100DB000CF910C94CF21C85AC73158F4EC2FF0E0F2
:100DC000EE0FFF1FEB57FF4F80819181CF910C9465
:100DD000E521CF910895882349F1682F8CEF860F84
:100DE000813A38F480916200909163000E943F2222
:100DF0000CC080E2860F883050F4677081E001C03B
:100E0000880F6A95EAF70E94270F0C94600F8BE514
:100E1000860F833020F480E090E00C94CF21685A54
:100E2000673120F480E090E00C94E52108951F9351
:100E3000CF93DF93182FEB010E949D06209741F07E
:100E400087EB9BE00197F1F700C000002197F6CFF8
:100E5000812FDF91CF911F910C94EB06893319F00C
:100E600060E070E002C060E570E00C941707882332
:100E700021F00E94210F0C94600F0895882321F027
:100E80000E94270F0C94600F0895CF92DF92EF928B
:100E9000FF920F931F93CF93DF937C01D62FC72F21
:100EA000FC011281058102950F700E94170F8823A3
:100EB000B9F01123A9F08C2F807F803421F080E2DB
:100EC0008D0F883068F080918A0282FD09C082E02F
:100ED0000E94C00F0E94170F91E0D82ED92601C0A2
:100EE000D12CCC2EC2948FE0C8228C2D90E08C3077
:100EF000910508F0C4C1FC01E65DFF4F0C943A2651
:100F00008C2F807FCF70882311F0C295C07F112372
:100F100099F0CC2309F49FC180E28D0F883010F046
:100F2000D11104C08C2F0E94210F03C08C2F0E946E
:100F3000310F0E94600F8FC18D2F0E94EB06CC23D2
:100F400009F49DC180E28D0F883038F1DD2329F14D
:100F50008C2F0E94370F24C08C2F807FCF7080325F
:100F600011F0C295C07FDD2319F0D130A1F13DC051
:100F700080918A0282FF17C0112349F0CC2329F007
:100F80008C2F0E94210F0E94600F80E065C180E0DD
:100F90000E94EB06CC2309F472C18C2F0E94270F0C
:100FA0000E94600F6CC1112371F0002341F00130E9
:100FB00031F40E94410F8C2B0E94490F60C10E94A6
:100FC000410F8C2B1DC0002319F0013009F457C1CB
:100FD0000E94560F25C0112321F0063008F04FC1A2
:100FE0000EC0053008F04BC11BC0112361F0002377
:100FF00031F0F701858180FF2EC18F7085838C2FA2
:101000000E9437073CC1002359F0D93309F034C19D
:10101000FFEF0DEE12E0F15000401040E1F72AC161
:101020008C2F0E943E072BC18C2F8695869583704E
:1010300019F0813061F023C1112321F08D2F9C2FF5
:10104000937002C080E090E00E94CF2120C1112364
:1010500021F08D2F9C2F937002C080E090E00E94C1
:10106000E52115C18C2F837009F047C011110BC108
:101070002D2F229526952770220F220F6D2F6F702E
:10108000862F90E0A0E0B0E0022E04C0880F991FE8
:10109000AA1FBB1F0A94D2F7D4FF10C04FE050E044
:1010A00060E070E004C0440F551F661F771F2A954B
:1010B000D2F7409550956095709503C040E050E0A0
:1010C000BA01C695C695C3708A019B01082B192BDE
:1010D0002A2B3B2BC901B801C23049F058F4C1306A
:1010E00019F00E94370ACFC00E94250ACCC00E9486
:1010F000490AC9C00E94230AC6C0112319F08C2FC7
:10110000817001C08695882309F4BDC02D2F2295DA
:1011100026952770220F220F6D2F6F70862F90E07B
:10112000A0E0B0E0022E04C0880F991FAA1FBB1FC9
:101130000A94D2F7D4FF10C04FE050E060E070E0B6
:1011400004C0440F551F661F771F2A95D2F740959C
:1011500050956095709503C040E050E0BA01C69587
:10116000C695C3708A019B01082B192B2A2B3B2B98
:10117000C901B801C23049F058F4C13019F00E94D9
:10118000FC0A81C00E94EA0A7EC00E940E0B7BC04E
:101190000E945D0A78C0CF70112339F08C2F0E9415
:1011A000830A8D2F0E9437076EC08D2F0E943E0745
:1011B0008C2F0E94A40A67C0D23F21F128F4D03FAF
:1011C00041F0D13FC1F043C0D33F19F1D43F79F092
:1011D0003EC0112341F0053008F051C08C2F8F71B3
:1011E0000E94C90A4CC0063008F049C0F7CF809170
:1011F0008A0282FF18C0112339F08C2F8F710E9450
:10120000830A3DC01123C9F38C2F8F710E94A40A59
:1012100036C0112329F08C2F8F710E946E0A2FC0C7
:101220000E94690A2CC0112349F0CF718C2F0E94B3
:10123000830A63E08C2F0E94A50F21C081E00E94E9
:10124000C00F0230E0F082E00E94C00F18C01123EE
:1012500031F0002391F28D2F0E949D0610C00023D3
:1012600099F2D93349F41FEF2DEE32E011502040AE
:101270003040E1F700C000008D2F0E94EB0688EFA0
:101280008C0D843020F40E94B8210E943206DD20AB
:10129000C9F00E94130F80FD15C0F70112820E9451
:1012A0000D0F0E94830AC7010E9483090E940D0F3F
:1012B000DF91CF911F910F91FF90EF90DF90CF9032
:1012C0000C94A40ADF91CF911F910F91FF90EF90A2
:1012D000DF90CF9008950F931F93CF93DF93EC018E
:1012E000688179818A810E94C50B8C010E94200B44
:1012F0000E94110AB801CE010E944507DF91CF91EB
:101300001F910F910895CF93DF93EC01988189810C
:101310002B813C81232B31F08F3F31F481E09F3FC3
:1013200019F403C081E001C080E080FD1DC0CE0142
:101330000E94BD05811110C00E94170F8823A1F0E3
:101340008A81882389F080918A0282FD0DC082E023
:10135000DF91CF910C94C00FCE010E946B09CE019A
:10136000DF91CF910C949E05DF91CF91089580E09D
:1013700090E00E94CF2180E090E00E94E5210E9451
:101380003E0F0C94600F80916200909163000E9468
:1013900041220C94B7090E942E0F0C94C309929518
:1013A0009F70963079F010F4925001C09A509230AC
:1013B00068F4803F69F018F4883E40F409C0843F27
:1013C00029F406C0883E20F0813F11F080E00895A6
:1013D00081E00895FC01808191810E94BA0B0E94F6
:1013E000CF090895CF93DF9300D000D01F92CDB7DF
:1013F000DEB70F900F900F900F900F90DF91CF916D
:101400000895CF93DF9300D000D000D0CDB7DEB7E2
:1014100026960FB6F894DEBF0FBECDBFDF91CF91F9
:101420000895089508950C94120A0C94130A0E94CA
:10143000150A60937001709371018093720190930B
:1014400073010C94B7090C94170A0F931F93009122
:101450007001109171012091720130917301602B24
:10146000712B822B932B1F910F910C94170A0F93C2
:101470001F930091700110917101209172013091C0
:10148000730160237123822393231F910F910C9486
:10149000170A0F931F930091700110917101209111
:1014A00072013091730160277127822793271F9162
:1014B0000F910C94170A0C94120A0E945B0A609315
:1014C0006C0170936D0180936E0190936F010C9489
:1014D000B70960E070E0CB010C945D0A0F931F9395
:1014E00041E050E060E070E08A019B0104C0000F21
:1014F000111F221F331F8A95D2F7C901B8011F910E
:101500000F910C945D0A0F931F9341E050E060E04F
:1015100070E004C0440F551F661F771F8A95D2F7ED
:1015200080916C0190916D01A0916E01B0916F015D
:101530008A019B01082B192B2A2B3B2BC901B801CF
:101540001F910F910C945D0A0F931F9341E050E09F
:1015500060E070E004C0440F551F661F771F8A9536
:10156000D2F7409550956095709580916C0190915F
:101570006D01A0916E01B0916F018A019B0108235A
:1015800019232A233B23C901B8011F910F910C9401
:101590005D0A0F931F9341E050E060E070E004C0EB
:1015A000440F551F661F771F8A95D2F780916C01F3
:1015B00090916D01A0916E01B0916F018A019B0124
:1015C000082719272A273B27C901B8011F910F9126
:1015D0000C945D0A0F931F9300916C0110916D01A3
:1015E00020916E0130916F01602B712B822B932B18
:1015F0001F910F910C945D0A0F931F9300916C0142
:1016000010916D0120916E0130916F016023712363
:10161000822393231F910F910C945D0A0F931F93C4
:1016200000916C0110916D0120916E0130916F015C
:1016300060277127822793271F910F910C945D0AD1
:1016400008952FE0929F800D1124E82FE695E695EE
:10165000E695877051E001C0550F8A95EAF785E05D
:10166000E89FF0011124EA5DFE4F20E030E070E0D9
:101670004081CB01022E02C0969587950A94E2F72D
:101680008170819584278523842781932F5F3F4F25
:101690002530310569F708952FE0929F800D1124C0
:1016A000682F669566956695982F977085E0689F78
:1016B000B001112440E050E080E0FB01E40FF51F91
:1016C000EA5DFE4F208130E0092E02C03695279555
:1016D0000A94E2F721703327042E01C0220F0A94E6
:1016E000EAF7822B4F5F5F4F4530510531F7089580
:1016F000BF92CF92DF92EF92FF920F931F93CF93FF
:10170000DF938C01C0906C01D0906D01E0906E0170
:10171000F0906F018091700190917101A091720120
:10172000B0917301C82AD92AEA2AFB2ACFE1D0E076
:10173000D701C6010C2E04C0B695A795979587953D
:101740000A94D2F780FD04C0219790F7B12C07C00E
:10175000BC2EB8018C2F0E94B9120197A9F38B2DD2
:10176000DF91CF911F910F91FF90EF90DF90CF907D
:10177000BF900895CF93DF93EC010E94780BBE01D8
:101780000E94B912DF91CF9108951F93CF93DF93F9
:10179000EB0190912501992321F0CB010E94BA0B16
:1017A00013C0882349F0CB010E94780B182F682FB3
:1017B000CE010E94210B04C0CB010E944C0B182FBC
:1017C000BE01812F0E94B912DF91CF911F91089520
:1017D0001F93CF93DF93C091740116E08091750140
:1017E000C81799F0D0E01C9FF0011D9FF00D112447
:1017F000EA58FE4F408151816281738184819581D5
:101800000E94010A2196C770E9CFDF91CF911F9105
:1018100008954091A6015091A7016091A80170918F
:10182000A9018091AA019091AB010C94010AEF9259
:10183000FF920F931F93CF93DF938091AB0182951B
:101840008F7009F065C08091A801882309F460C0F9
:1018500080917401F09075011091A6010091A7018B
:101860006091A9017091AA0191E01F3F09F090E0F9
:10187000C0916000D0916100292F96E0E92E8F156C
:1018800009F446C06115710521F00F3F21F030E0E9
:1018900003C031E001C0322F90E030FD36C0E89E39
:1018A000F001E99EF00D1124DF01AA58BE4F1196F8
:1018B0003C911197301329C03C91311326C01296E8
:1018C0003C911297311121C013964D915C91149760
:1018D000461B570B4C175D07C0F48091AB018F700E
:1018E00080618093AB01E558FE4F80818F708061ED
:1018F000808386EA91E00E948309DF91CF911F9156
:101900000F91FF90EF900C94E80B01968770B7CF82
:10191000DF91CF911F910F91FF90EF9008959F92CB
:10192000AF92BF92CF92DF92EF92FF920F931F93ED
:10193000CF93DF93CDB7DEB761970FB6F894DEBFD4
:101940000FBECDBF8C0185E0F801DE011D96019030
:101950000D928A95E1F7D8011296EC909091A6012C
:10196000E091A7012091A9013091AA01211531052B
:1019700031F0EF3F31F481E09F3F19F403C081E083
:1019800001C080E0B82FB1709B2E80FD47C1D80107
:101990004C9111965C9111971396AD90BC90149751
:1019A00086EAC82E81E0D82EF090A801B501621B0E
:1019B000730B2091600030916100FF2009F4D9C0C1
:1019C0008091AB016217730708F095C0282F207F24
:1019D00009F052C05E1313C0491311C0FE2CE11070
:1019E0000EC08F7080618093AB010E94090CC6010C
:1019F0000E9483098091AB01F80185834DC1AB281A
:101A000031F05F3F31F481E04F3F19F403C081E0D2
:101A100001C080E080FD03C081E08E2502C080E02F
:101A200090E0F82FF170FF2E80FF1CC080917401B0
:101A30002091750136E0821709F40BC190E0389FC0
:101A4000F001399FF00D1124EA58FE4F61815613C1
:101A500006C06081461303C06281E61203C001968E
:101A60008770E9CFFE2CEE2009F416C18091AB01FE
:101A700081608093AB0154C05E1306C0491304C05B
:101A8000E11002C0F80199C0C8010E94EA09882348
:101A900061F1EE2051F12091AB01822F82958F7080
:101AA00090E0029774F08091A6019091A701988729
:101AB0008F831986BB86AA862C87CE0107960E9443
:101AC000830986E0F801A6EAB1E001900D928A95BB
:101AD000E1F70E94170C0E94090C0AC05E1711F171
:101AE000C8010E94EA0981112CC0C8010E94830923
:101AF000FF24F394D1C0282F207F81F77A2DB98A53
:101B0000A88A6E2D89890E94F20986EA91E00E94D6
:101B1000830986E0D6011D928A95E9F70E94090C97
:101B2000F12CBAC04913DCCFE110DACFF80185837C
:101B3000C8010E94830986E0D6011D928A95E9F7C3
:101B4000ABC0EE2091F22091AB01822F82958F7075
:101B500090E002970CF4B5CF8091A6019091A70177
:101B60009A8389831B82BD82AC822E83CE0101962B
:101B7000A6CF6217730708F044C0FE2CEE2009F4CC
:101B8000B4CF5E1330C049132EC02091AB0120FDAD
:101B900021C0822F82958F70482F50E0411551054A
:101BA000C9F0F80125834F30510541F08F5F982F20
:101BB0009295907F822F8F70892B8583C8010E9418
:101BC000830986E0F801A6EAB1E001900D928A95BA
:101BD000E1F73CC086E0F801A6EAB1E001900D9281
:101BE0008A95E1F759C0C8010E94EA09811169CFBD
:101BF0008091AB0181608093AB01C8010E94830991
:101C00004BC07A2DB98AA88A6E2D89890E94F20963
:101C100086E0D6011D928A95E9F718C0EE2009F4F6
:101C200064CFC8010E94EA09F82E882309F45DCF29
:101C300086E0F801A6EAB1E001900D928A95E1F7FD
:101C400086EA91E00E9497060E94170C0E94090CF8
:101C500023C04D875E878D859E850E94BA0B292FF4
:101C600022952F70223028F49F7039F0811105C021
:101C70000BC0243028F49F7049F4805E883020F037
:101C8000C8010E9483099F2CF92C06C0D801159623
:101C90009C91907F91F7F8CF8F2D61960FB6F894B5
:101CA000DEBF0FBECDBFDF91CF911F910F91FF908F
:101CB000EF90DF90CF90BF90AF909F9008951F93CB
:101CC000CF93DF93CDB7DEB72C970FB6F894DEBF76
:101CD0000FBECDBF4F83588769877A878B879C87D4
:101CE000CE0107960E948F0C8823D1F09F818885B2
:101CF0002A853B85232B31F08F3F31F481E09F3FD4
:101D000019F403C081E001C080E080FD47C04F812D
:101D1000588569857A858B859C850E94010A3EC01D
:101D200086E0FE013796DE01119601900D928A95AC
:101D3000E1F7FF81E8856A857B856115710531F0E2
:101D4000EF3F31F481E0FF3F19F403C081E001C0AF
:101D500080E080FD23C02091750130E0C90101962B
:101D6000877099274091740150E084179507F1F12D
:101D7000F983EA837D836C8396E0929FD001939FE1
:101D8000B00D1124AA58BE4FFE01319601900D925C
:101D90009A95E1F7809375010E94E80B16E0809117
:101DA000740190917501891771F1189FC001112478
:101DB0008A589E4F0E948F0C882329F1E09174016C
:101DC0001E9FF0011124EA58FE4F4081518162812B
:101DD0007381848195810E94010A8091740190E051
:101DE00001968770992780937401D9CF0E94CB09FF
:101DF0001092750110927401E6EAF1E086E0DF01CD
:101E00001D928A95E9F72C960FB6F894DEBF0FBEA7
:101E1000CDBFDF91CF911F9108958091B401859539
:101E20008595859508958091B40187700895909166
:101E3000B401977081E009F480E008958091BF01BA
:101E400008959091BF01892B8093BF0108958095DB
:101E50009091BF0189238093BF0108951092BF0123
:101E600008959091BE01892B8093BE0108958095BD
:101E70009091BE0189238093BE0108951092BE0106
:101E800008958091B501089508950C94440F0C9421
:101E9000450F90918A0292FD08C09091B501981764
:101EA00021F08093B5010C94470F08958091B501FE
:101EB000882329F01092B50180E00C94470F089513
:101EC000CF93DF93E0916200F09163008091BF01B6
:101ED0008083E0916200F091630090818091BE0167
:101EE000892B80838091B501882381F0E091620085
:101EF000F09163009081892B8083809162009091A2
:101F000063000E94FB2181110E94560FC091620064
:101F1000D091630048E050E06CEA71E0CE010E948D
:101F20008A26892B69F088E0FE01ACEAB1E00190D5
:101F30000D928A95E1F7CE01DF91CF910C94C421E7
:101F4000DF91CF9108950C94440F90918A0292FDF5
:101F500010C098E0899F90011124262B2093B40192
:101F60000E94830A8091B4018595859585950C948E
:101F7000A30F0C94830A1092B40180E00C94A30F79
:101F80002091B401809582238093B401982F97709B
:101F900099F430E0482F082E000C550B2417350714
:101FA00059F090918A0292FD07C085958595859597
:101FB0000E94A40A0C94BB0F089590918A0292FB90
:101FC000222720F9281769F080FB92F990938A0262
:101FD0008091890290918A020E942B1082E00C94D9
:101FE000C00F089580918A0282FB882780F991E0D2
:101FF00089270C94DD0F81E00C94DD0F80E00C94B8
:10200000DD0F6FEF7FEF80E090E00C94C82680E05A
:1020100090E00E94A52621E0893E9E4F09F020E035
:10202000822F089582E090E00C94972683E090E060
:102030000C949726CF9384E090E00E949726C82FB7
:1020400082E290E00E9497262C2F30E0A901582BC5
:10205000CA01CF910895CF93C92F682F84E090E0F3
:102060000E94AB266C2F82E290E0CF910C94AB26BD
:10207000AB01BC018FE090E00C94BC26AB01BC012D
:1020800083E190E00C94BC2660E070E0CB010C94FE
:102090003E1060E070E0CB010E9438100C944410B8
:1020A00069EE7EEF80E090E00E94C82660E082E06A
:1020B00090E00E94AB2660E083E090E00E94AB26B7
:1020C00010927001109271011092720110927301BE
:1020D00060E084E090E00E94AB2660E082E290E065
:1020E0000E94AB2660E085E090E00E94AB2660E0B5
:1020F00086E090E00E94AB266FEF87E090E00E94C0
:10210000AB2640E050E0BA0188E090E00E94BC2697
:1021100060E08DE090E00E94AB2640E050E0BA0124
:1021200088E190E00E94BC2660E087E190E00E9498
:10213000AB2640E050E0BA018CE190E00E94BC2662
:1021400060E070E080E290E00E94C82640E050E04D
:10215000BA0188E190E00E94BC260C9449100C94CE
:102160005010682F8EE090E00C94AB260E948622DF
:102170006093D2017093D3018093D4019093D501E1
:102180006093CE017093CF018093D0019093D101E1
:10219000089584B7806884BF84B7806884BF089539
:1021A00081E008950C94D01008950C94D4100C94F0
:1021B000D4100C94D7100C94D4100C94DB100C9405
:1021C000D4100E94C91085E993E10E94AE210E94BB
:1021D000DF100C94DD100E94D5100C94D4100E94D6
:1021E000B2130E9431060C946D1E0E9473220E944D
:1021F00097140E94EF100E94571C0E94961A0C948C
:10220000D9105F926F927F928F929F92AF92BF92FE
:10221000CF92DF92EF92FF920F931F93CF93DF93B2
:10222000CDB7DEB72A970FB6F894DEBF0FBECDBF8D
:102230000E94AC14C82E81110E94B61030EC832E7F
:1022400031E0932E00E010E0502E802F0E94D61334
:102250005C01F401619071904F0168267926611448
:102260007104B1F40F5F1F4F0730110569F78FEF4D
:1022700089838A831B820E947A228160782F9D83C2
:102280008C8349815A816B818D810E944D063AC0B1
:102290008091D60181FD0E94DF13D12CEE24E394BE
:1022A000F12CC3018E219F21892B29F10E94D2108C
:1022B0008823A9F0DE825F82AE20BF2081E0AB28B8
:1022C00009F480E088870E947A228160782F9A87BB
:1022D00089874E815F8168858A850E944D06000F3F
:1022E000111FF801E054FE4F80819181E826F92604
:1022F000F182E08207C0D394EE0CFF1CFFE0DF12F6
:10230000D0CFB0CF81E0C11001C080E02A960FB6D7
:10231000F894DEBF0FBECDBFDF91CF911F910F911B
:10232000FF90EF90DF90CF90BF90AF909F908F90F5
:102330007F906F905F9008950E9401110E94C91ACA
:102340000E946C1E0C944206CF93DF930E94BE1233
:10235000EC01811522E59207E8F5811531E5930737
:1023600008F0B6C0883E910528F5803E910508F03A
:10237000E9C0883A910570F4853A910508F07AC071
:102380008130910509F473C008F4D9C0049708F0AE
:10239000D9C0D5C08F3B910508F0D1C0C85AD0E054
:1023A000CC0FDD1FCA54DF4F0990D881C02DCE015C
:1023B0009464C9C0811540E5940708F069C081158F
:1023C00050E4950708F060C09A9581159F4108F484
:1023D000B9C0B5C0811536E5930728F5811545E5E7
:1023E000940708F092C0811554E5950708F087C05E
:1023F000AC0143705527282F26952695C115D34546
:1024000008F06CC081E090E002C0880F991F4A95E7
:10241000E2F740E2249F90011124EC01C22BD32B60
:10242000CE019C6890C081152AE5920780F4811541
:1024300039E5930708F072C0811548E5940708F460
:102440007EC0D82FCC27CE01806F906A7CC090567A
:102450008115904208F073C08D2F8F710E94521326
:10246000DD27D0628F71AE01582BCA016CC081E0AC
:1024700090E069C0C55AD0E0CC51DF4F8881C82FA9
:10248000D0E0CE0190645FC0DF70CE01906A5BC087
:1024900074E0969587957A95E1F7282F23703C2F65
:1024A000337081E090E002C0880F991F3A95E2F7FF
:1024B0009C68AC01522B9A019C2F9F709695969523
:1024C00050E2959FE0011124C9018C2B9D2B3BC04C
:1024D000D82FCC27CE01816F906A35C081E090E083
:1024E00002C0880F991F4A95E2F750E2259F90019C
:1024F0001124EC01C22BD32BCE019A6824C0D82F13
:10250000CC27CE01846F906A1EC00E9452138F7137
:1025100090E0D82FCC27CE01906215C08F700E941A
:10252000521394E0D695C7959A95E1F7CF70D0E015
:10253000DC2FCC27D0699E01282BC90104C080E084
:1025400090E001C0CE01DF91CF91089529E6829FEE
:10255000C0011124FC012FE0729FE00DF11D112438
:10256000E60FF11DEE0FFF1FE459FF4F8591949187
:1025700008950E94A6120E94A41108958238910520
:1025800069F1B0F48133910509F46DC048F48932E2
:10259000910509F463C08A32910509F469C0089570
:1025A0008533910509F455C089339105B9F0089533
:1025B000833E910569F138F4803E9105B1F0823E89
:1025C000910509F10895863E9105A9F1873E91058F
:1025D000B9F1843E910509F064C023C020918902BD
:1025E00020FD4FC021FD4DC008958091890280FDDE
:1025F00044C080918A0280FF44C08091890284FD9A
:1026000042C083EE4DC08091890282FF38C0F5CF71
:102610008091890282FD33C080918A0280FD31C0A1
:10262000ECCF80918A0281FF32C08091890284FDC3
:102630002AC087EE35C08091890283FF26C0F5CF7E
:102640008091890283FD21C080918A0281FD1FC093
:10265000ECCF8091890285FD1CC01DC0809189024C
:1026600085FD19C016C08091890286FD16C017C06D
:102670008091890286FD13C010C089E311C082EEEB
:102680000FC080EE0DC080E00BC086EE09C084EE66
:1026900007C089E205C085E303C08AE201C081E387
:1026A00090E008959091890292FF0DC0282F287123
:1026B000283019F4877F846006C0282F24712430C5
:1026C00011F48B7F886093FF0DC0282F287128316B
:1026D00019F4877E846106C0282F2471243111F4F7
:1026E0008B7E886120918A0220FF0DC0382F3871BF
:1026F000383019F4877F816006C0382F317131304E
:1027000011F48E7F886021FF0DC0282F2871283199
:1027100019F4877E816106C0282F2171213111F4BF
:102720008E7E886194FD877E089580E008950C94E4
:1027300001100E94AC142FE389E191E02150804008
:102740009040E1F700C000000E94AC1480E00E94BD
:10275000D61380FF04C00E9497130C94C7220895DB
:102760000C9499130E940710811102C00E94AF10AF
:102770000E9412108093D6010E941A1090938A0230
:10278000809389020E94B0130E941610682F70E097
:1027900080E090E00E94230A60916C0170916D01CD
:1027A00080916E0190916F010C945B0AE82FF0E02C
:1027B000EE0FFF1FE756FD4F808191810895089528
:1027C00088E78A95F1F7089500C008950C94E01306
:1027D00008950C94E8130C94E9130C94E8130C94EA
:1027E000ED13F894E82FE295EF70F0E031A9282F6F
:1027F0002F7081E090E001C0880F2A95EAF7982FAA
:102800009095932391AB92A9892B82AB78940895EC
:102810000F931F93CF93DF93C6EFD0E089918F3F43
:1028200011F00E94F11380E0CD3FD807B9F7C7EE51
:10283000D0E006EF10E089918F3F11F00E94F11374
:102840000C171D07C1F7DF91CF911F910F910895CC
:10285000BF92CF92DF92EF92FF920F931F93CF938D
:10286000DF938C01C62FD0E0CE018A509F4F6C01C0
:10287000FC0190819F3F09F450C0B62EF894E92FD7
:10288000E295EF70F0E081A99F7021E030E001C097
:10289000220F9A95EAF7822B81AB82A920952823F3
:1028A00022AB78940E94E413E7EEF0E046EF50E0AC
:1028B00021E030E0E12CF12C61916F3F89F0A62FEF
:1028C000A295AF70B0E0D0968C9190E06F7002C08E
:1028D000959587956A95E2F780FD02C0C90102C00F
:1028E00080E090E0E82AF92A220F331F4E175F0795
:1028F00019F7F60180818F3F11F00E94F11361E01A
:10290000E114F10409F460E08B2D0E94E613CC0F72
:10291000DD1FC00FD11FF982E882DF91CF911F9197
:102920000F91FF90EF90DF90CF90BF9008950E949D
:1029300008148EE0E9E9F2E0DF01982F1D929A95E4
:10294000E9F7EBE8F2E0DF011D928A95E9F787E00D
:102950000E94F7140C94A905FF920F931F93CF9335
:10296000DF93CDB7DEB72E970FB6F894DEBF0FBE5C
:10297000CDBF8E010F5F1F4F8EE0F80111928A9537
:10298000E9F7F12C6F2DC8010E942814F394F7E0A9
:10299000FF12F8CF4EE050E0B8018BE892E00E94C1
:1029A0008A26FF24F394009709F4F12C892B41F037
:1029B0008EE0F801ABE8B2E001900D928A95E1F764
:1029C0002F2D47E069E972E08BE892E00E94F8144D
:1029D0000E94AB058F2D2E960FB6F894DEBF0FBE6A
:1029E000CDBFDF91CF911F910F91FF900895089572
:1029F000FF920F931F93CF93DF93F82E092F162F7B
:102A0000D72FC42F222349F081E08093D9010E945F
:102A10007A229093D8018093D7018091D90188239D
:102A2000D9F08091D7019091D8010E949222059708
:102A300098F0EF2DF02FA12FBD2F80E090E04C2FCC
:102A400050E08417950734F4219131912D933D93F3
:102A50000196F7CF1092D901DF91CF911F910F917D
:102A6000FF9008950E94DC220E94F5100C94ED2244
:102A70000E9468220E94D5220E94E1100E94321515
:102A80000E94FB220E94EB10FBCFEF92FF920F936C
:102A90001F93CF93DF938B01682F11110AC044233A
:102AA00029F0E82FF0E0E356FA4F6491762F862F55
:102AB00075C0212F30E0E82FF0E0442321F0E356E9
:102AC000FA4FE491F0E046E0049FC0011124CFEFFB
:102AD000D0E0BE010E94F0254BEA4603C001479FAB
:102AE000900D1124800F911D800F911D982F990F2B
:102AF000890FAE01421B530B4E9FD0014F9FB00D6B
:102B00005E9FB00D11249B2F189FA0011124452F0B
:102B100055278E01041B150B0E9FA0010F9F500D12
:102B20001E9F500D11247E01E81AF108E29E8001DB
:102B3000E39E100DF29E100D1124212F3327C21B8E
:102B4000D30BCE9F9001CF9F300DDE9F300D11240F
:102B500062307105A9F048F46115710569F06130C2
:102B60007105C9F48B2F752F0DC06430710581F08C
:102B700058F06630710579F47E2F8B2F932F0DC09E
:102B8000832F7B2F9E2F09C08E2F7B2F952F05C063
:102B90008E2F732F02C07E2F852F692FDF91CF914B
:102BA0001F910F91FF90EF90089541E00E9445150D
:102BB000089508950E94D5150895CF93DF93762F39
:102BC000E901682F842F0E94DA15798368838A834C
:102BD000DF91CF9108958091A702282F269530E0AC
:102BE0002115310519F48170826005C02532310547
:102BF00024F0817088648093A702089588E090E0B3
:102C00000C949F26CF92DF92EF92FF926B017C0192
:102C10000E94EB15B701A60188E090E0FF90EF90CD
:102C2000DF90CF900C94BC26E7EAF2E083E080834B
:102C300011828FEF8283838314826081718182810C
:102C400093810C9402168091A70280FF02C08695A2
:102C5000089580E008959091AB02933018F49F5F3F
:102C60009093AB02882351F06091A7027091A80263
:102C70008091A9029091AA020C940216089581E015
:102C80000C942B169091AB02992319F091509093CC
:102C9000AB02882351F06091A7027091A802809145
:102CA000A9029091AA020C940216089581E00C9456
:102CB000421670E00C94791E609168008091A70222
:102CC00080FF0AC08091670023E0829FC001112429
:102CD00084559D4F0C9459168091690090916A001B
:102CE000891780F7E82FF0E09F01220F331FE20FD2
:102CF000F31FE455FD4F1182108212828F5FF0CFD7
:102D00009091A70290FF16C09091690020916A00EF
:102D1000921770F4E92FF0E0DF01AA0FBB1FEA0F52
:102D2000FB1FE455FD4F8183608342839F5FF0CF9B
:102D30000C945C160895CF93DF9300D01F92CDB70B
:102D4000DEB79091A70290FF0AC09E012F5F3F4F10
:102D50000E94DD154B8169818A810E9480160F9047
:102D60000F900F90DF91CF910895CF93DF93EC01F7
:102D7000EC81F0E0E856FB4F4491E7EAF2E0628133
:102D800081810E949B168C818F5F8C83DF91CF9114
:102D90000895CF93DF93EC01E7EAF2E0438162818B
:102DA0008C810E949B168C818F5F8C83DF91CF91E9
:102DB00008950F931F93CF93DF9300D01F92CDB749
:102DC000DEB78C018091DA0181110AC09E012F5F6C
:102DD0003F4F4FEF6FEF0E94DD158A818093DA013C
:102DE000F8018481813051F028F0823061F4409103
:102DF000DA010AC08091DA0140E007C06091DA018F
:102E000040E080E003C040E080E060E00E94801687
:102E1000F801848190E0019663E070E00E9404264E
:102E200084830F900F900F90DF91CF911F910F919E
:102E30000895AF92BF92CF92DF92EF92FF920F93DD
:102E40001F93CF93DF9300D01F92CDB7DEB7182F1B
:102E5000F62E042FE22E9091A70290FF6DC0E92F6D
:102E6000E695AE2FB0E0A350BF4F8C918093E40164
:102E70009E7F923061F49E012F5F3F4F812F0E9411
:102E8000DD154B8169818A810E94801643C08230A2
:102E900019F40091AA023EC0863019F41091A802DC
:102EA00039C08930D9F38931A9F5E9518E2F817064
:102EB000D82EE695F0E0E856FA4FA590B490C12CD4
:102EC000BB2460916B00C61618F52C2D30E0A29E35
:102ED000C001A39E900DB29E900D112470E00E943F
:102EE000F025812FD11002C0860F01C0861B909162
:102EF0006900290F311DA901440F551F240F351FEB
:102F000024553D4F402F6F2D0E94DD15C394D9CF1E
:102F10000E945C161093A802F092A9020093AA02E4
:102F2000EE2051F06091A7027091A8028091A90251
:102F30009091AA020E9402160F900F900F90DF91BD
:102F4000CF911F910F91FF90EF90DF90CF90BF90A6
:102F5000AF900895E7EAF2E09181282F43816281E2
:102F60008CE0890F0C94191781E00C94AA17E7EAFA
:102F7000F2E09181282F4381628184EF890F0C94C4
:102F8000191781E00C94B717E7EAF2E062812FE0AD
:102F9000620F08F46FEF282F438181810C94191779
:102FA00081E00C94C417E7EAF2E062812FE0621B33
:102FB00008F460E0282F438181810C94191781E087
:102FC0000C94D317E7EAF2E0438122E1420F08F4C0
:102FD0004FEF282F628181810C94191781E00C94A6
:102FE000E217E7EAF2E0438122E1421B08F440E005
:102FF000282F628181810C94191781E00C94F117BC
:1030000020E00C941917FF920F931F93CF93DF9337
:10301000EC01F12C0FEF10E060916B00F616F0F46C
:10302000809169002F2D30E0280F311DC901880FD4
:10303000991F280F391F24553D4F70E0C8010E9489
:103040000426962F8C814091AA026091A902F99ED4
:10305000800D11240E94DD15F394DECF0E945C16D2
:103060009A818C8190FF02C08F5F01C081508C8358
:10307000DF91CF911F910F91FF900895AF92BF9272
:10308000CF92DF92EF92FF920F931F93CF93DF9334
:10309000FC01828180FF02C00FEF01C001E010E05F
:1030A0004CE0A42E80916B00181708F043C080916B
:1030B0006900C12ED12CE601C80FD11DCE01880FA9
:1030C000991FC80FD91FC455DD4F198218821A8263
:1030D00034E0E32EF12CB12C8091DC018B0D8D308E
:1030E0002CF06A2D0E94E225892F05C087FF03C0BE
:1030F00090916B00890F082E000C990BC816D90609
:1031000091F48091AA028E9DA0018F9D500D1124F3
:1031100055954795559547959E016091A9028091D7
:10312000A8020E94DD15B00EF1E0EF1AF108A1F639
:103130001F5FB8CF0E945C168091DC01013031F432
:10314000811102C080916B00815007C090E0019610
:1031500060916B0070E00E9404268093DC01DF9197
:10316000CF911F910F91FF90EF90DF90CF90BF9084
:10317000AF900895CF938091690090916A0089176C
:1031800070F4E82FF0E09F01220F331FE20FF31FCE
:10319000E455FD4F1182108212828F5FF0CFC0E0A4
:1031A00060916B00C617C0F5EC2FF0E070E0CF0126
:1031B0000E94042620916900820F2091DB01022EDB
:1031C000000C330B90E0E217F307CCF0209166007F
:1031D000022E000C330B2E173F078CF09C01220FA0
:1031E000331F820F931F9C0124553D4F4091AA022B
:1031F0006091A9028091A8020E94DD150BC0FC011C
:10320000EE0FFF1F8E0F9F1FFC01E455FD4F118233
:1032100010821282CF5FC4CF0E945C16209165009D
:103220008091DB01820F8093DB0190916600920F09
:103230009093660019165CF4082E000C990B4091CF
:103240006B0050E041505109841795071CF02195FF
:1032500020936500CF9108958F929F92AF92BF9275
:10326000CF92DF92EF92FF920F931F93CF93DF9352
:103270008C01FC014481C42FD0E09E01DE010E943C
:1032800048269B01AC010E945E266B017C01E0E2B6
:10329000F0E0EC1BFD0BA5E5B0E09B01AC010E944A
:1032A0005E264B015C019F01DF010E9440269B01CD
:1032B000AC010E9469269B01AC012C0D3D1D4E1DE9
:1032C0005F1DC501B4010E941826C22FD22F2A32D9
:1032D00028F4F3E02F9F900111240DC025E530E084
:1032E0002C1B3109C901880F991F280F391F37FF7F
:1032F00002C02F5F3F4F35952795C22FC095F12C07
:1033000085E5E82EED1A80916B00F816C8F4F1FC03
:1033100002C08E2D01C08D2F909169002F2D30E0BD
:10332000290F311DA901440F551F240F351F2455A6
:103330003D4F4C2F6091A9020E94DD15F394E3CF1D
:103340000E945C16F8018481811102C091E003C0E3
:10335000803219F49FEF9093640090916400890F7C
:10336000F8018483DF91CF911F910F91FF90EF902F
:10337000DF90CF90BF90AF909F908F9008950F9364
:103380001F93CF93DF93EC0100E010E080916B007E
:10339000282F30E00217130724F590916900980157
:1033A000290F311DA901440F551F240F351F245526
:1033B0003D4F869590E04C81081719071CF4442373
:1033C00031F002C0411103C04091AA0201C040E0A7
:1033D0006091A9028091A8020E94DD150F5F1F4F26
:1033E000D5CF0E945C168C8190E001968170992760
:1033F0008C83DF91CF911F910F910895E7EAF2E05E
:1034000080818E7F808360817181828193810E941F
:1034100002161092E5012FEB84ED91E021508040DF
:103420009040E1F700C000000C945C166091A70288
:10343000669570E04BE050E08CE690E00E947D26BF
:10344000892B19F481E08093E5010E947A22909300
:10345000DE018093DD0108959091A70290FF35C0B1
:103460009170811102C0926006C0853210F098649C
:1034700002C0880F982B9093A702662351F06091A9
:10348000A7027091A8028091A9029091AA020E94BD
:1034900002166091A702669570E04BE050E08CE662
:1034A00090E00E947D26892B19F01092E50102C060
:1034B0000E94161A81E08093E0014091AA02609177
:1034C000A9028091A8020C9400180895682F909189
:1034D000A702969581E0890F853208F081E00C946F
:1034E0002C1A81E00C94661A682F9091A702969589
:1034F0008FEF890F09F484E20C942C1A81E00C946C
:10350000741A61E00C942C1AE7EAF2E08081816081
:10351000808386950C94811A8091A70280FD0C947B
:10352000FE190C94841A60E00C942C1A8091E3012B
:1035300081112EC00E940710811104C00E94AF109B
:103540000E9414160E94FE156093A7027093A802B1
:103550008093A9029093AA026E7F61F40E941416D0
:103560000E94FE156093A7027093A8028093A9029F
:103570009093AA020E94EB151092E5018091A70298
:1035800080FF03C086950E94931A81E08093E30137
:1035900008950F931F93CF93DF938091E5018823C4
:1035A00009F485C08091E401E091A702E695E81B4B
:1035B000E093DF01823049F4F0E0EC56FB4FE491F8
:1035C000CE2FD0E005EB16E149C0863049F4F0E09B
:1035D000EF56FB4FE491CE2FD0E009EC16E13EC050
:1035E000893051F4E695F0E0E257FB4FE491CE2F9D
:1035F000D0E003E018E132C08F3051F4E695F0E0FE
:10360000E557FB4FE491CE2FD0E00EE318E126C042
:10361000853149F4F0E0E857FB4FE491CE2FD0E03C
:103620000AEB18E11BC0883181F0833239F4E6E8F7
:10363000F4E0C591D49109ED16E110C0843251F443
:10364000C4EFD1E00FEB19E109C0C8E2D0E00CE211
:1036500019E104C0C0EDD7E009ED15E18091E0016A
:10366000882361F01092E0010E947A229093DE019B
:103670008093DD011092E2011092E1010E947A2212
:10368000E091DD01F091DE018E1B9F0B8F3F9F4784
:1036900070F4EC0FFD1FF093DE01E093DD018DED82
:1036A00091E0F801DF91CF911F910F910994DF9183
:1036B000CF911F910F910895882311F0FA0101C055
:1036C000FB010994CF93DF93C82FD62F0E942316B6
:1036D0008C1740F00E9423168D1720F4DF91CF91B4
:1036E0000C94711A8C2FDF91CF910C94811A1F9337
:1036F000CF93DF93FB0112811111C3C0EC010E9433
:103700001E0F8272CD3CFCE5DF0709F49AC0A8F5D4
:10371000C73CECE5DE0709F476C0A8F4C43C9CE5A0
:10372000D90709F45FC028F4C33CDC4509F457C04D
:1037300054C0C53C9CE5D90709F459C0C63CDC45DA
:1037400009F45CC04AC0CA3CFCE5DF0709F46AC062
:1037500050F4C83CECE5DE0709F45AC0C93CDC452E
:1037600009F45BC03AC0CB3C9CE5D90709F45FC0C3
:10377000CC3CDC4509F460C030C0C23DFCE5DF074D
:1037800009F46FC088F4CF3C9CE5D90709F460C008
:1037900008F45CC0C03DFCE5DF0709F45CC0C13D36
:1037A000DC4509F45BC019C0C53D9CE5D90709F4A7
:1037B00060C050F4C33DFCE5DF0709F455C0C43DCB
:1037C000DC4509F454C009C0C63D9CE5D90709F49D
:1037D00055C0CE35DD4509F454C011E052C00E94F9
:1037E0008C1A4FC04EE75AE161E77AE104C041E725
:1037F0005AE16EE77AE10E945C1B43C041EC57E15D
:1038000064EB77E1F8CF44EB57E161EC77E1F3CF7C
:103810004FED57E160ED77E1EECF40ED57E16FED11
:1038200077E1E9CF4DEF57E16EEE77E1E4CF4EEE71
:1038300057E16DEF77E1DFCF46E556E16FE376E1E3
:10384000DACF4FE356E166E576E1D5CF81E017C0E8
:1038500065E082E010C068E086E00DC06EE089E0BF
:103860000AC064E18FE007C067E185E104C088E138
:1038700006C062E289E10E94621B03C083E20E94EB
:10388000811A812FDF91CF911F91089586E090E0FA
:103890000C949726682F86E090E00C94AB268091DC
:1038A000D002847089618093D0020C944A1C0E94DB
:1038B0000710811104C00E94AF100E944F1C0E948B
:1038C000461C8093D002282F26952695269530E019
:1038D0002430310524F0877088618093D002809174
:1038E000D00280FF04C086958695869501C080E051
:1038F0000C94BF1D2091D002822F869586958695C7
:10390000482F50E04330510554F48F5F982F990FA2
:10391000990F990F822F8770892B8093D002809105
:10392000D00281608093D0020E944A1C8091D00214
:103930008695869586950C94BF1D8091D002982F10
:10394000969596959695A1F0915E990F990F990F7E
:103950008770892B8093D002887F91E009F490E0F2
:103960008091D00290FB80F98093D0020E944A1C83
:103970008091D0028695869586950C94BF1D809186
:10398000D00280FD13C081608093D002813019F491
:1039900089E08093D0028091D0020E944A1C8091DD
:1039A000D0028695869586950C94BF1D08958091CA
:1039B000D00280FF08C08E7F8093D0020E944A1CF4
:1039C00080E00C94BF1D08958091D00280FD0C947E
:1039D000D71C0C94BF1C9091D002892F8695869598
:1039E00086958F5F8F719770843038F4880F880FB9
:1039F000880F892B8093D00202C09093D0028091CF
:103A0000D002887F91E009F490E08091D00290FB91
:103A100080F98093D0020E944A1C8091D002869542
:103A2000869586950C94BF1D843008F083E09091B4
:103A3000D0029770282F220F220F220F922B9093E3
:103A4000D002987F21E009F420E09091D00220FB81
:103A500090F99093D0020C94BF1D0E94141D809188
:103A6000D0020C944A1C9C01FB018281882349F1FD
:103A70002E3BFCE53F07C9F040F42C3BECE53E074C
:103A800069F02D3B3C4561F00895203C9CE53907E9
:103A900091F070F0213C3C4589F0089583E001C02D
:103AA00080E00E942D1D80E008950E949D1CFBCFA8
:103AB0000E947A1CF8CF0E94E41CF5CF0E94EB1CF8
:103AC000F2CF81E008958A9A92980895929A089583
:103AD000929808951F920F920FB60F9211242F9370
:103AE0003F934F935F936F937F938F939F93AF9386
:103AF000BF93EF93FF930E94681DFF91EF91BF91D9
:103B0000AF919F918F917F916F915F914F913F9175
:103B10002F910F900FBE0F901F9018951F920F922C
:103B20000FB60F9211242F933F934F935F936F9390
:103B30007F938F939F93AF93BF93EF93FF932AB598
:103B40003BB586B597B56AEF70E00E94F0256B5FD4
:103B50007F4F6217730710F40E94661DFF91EF916B
:103B6000BF91AF919F918F917F916F915F914F9195
:103B70003F912F910F900FBE0F901F9018958F922D
:103B80009F92AF92BF92CF92DF92EF92FF920F93EC
:103B90001F93CF93DF93C82F843078F481110EC028
:103BA0008AB59BB5892B31F089B78F7E89BF89B7DC
:103BB0008B7F89BF0E94681D0BC0C3E08AB59BB58F
:103BC000892B31F489B7806189BF89B7846089BF47
:103BD000A6B5B7B52C2F30E00E94482623E030E090
:103BE00040E050E00E9418260027122F232F342F88
:103BF000012F122F232F332786B597B56CE070E085
:103C00000E94F0256017710730F0C80169E070E08C
:103C10000E94F02552C086B597B5E6B4F7B4E6B574
:103C2000F7B5C6E0D0E0BE010E94F025060F171FD1
:103C3000211D311D4801590185E0880C991CAA1CE1
:103C4000BB1C8A95D1F7C701BE010E94F0256F0108
:103C5000E12CF12CA7019601260F371F411D511DA4
:103C6000C501B4010E94182669017A01E6B5F7B5CD
:103C7000CA01B9010E94D2259B01AC01DF010E945B
:103C80005E269B01AC01C701B6010E94D225DC0172
:103C9000CB012FE0B695A795979587952A95D1F7F3
:103CA00006B517B520E030E0081719072A073B07CB
:103CB00018F466B577B5CB01BC017BBD6ABDDF9159
:103CC000CF911F910F91FF90EF90DF90CF90BF9019
:103CD000AF909F908F90089508950E94631D82E099
:103CE0008FBD89E18EBD8FEF9FEF97BD86BD0C9490
:103CF000571C0F931F93CF93DF938C01EB0180919F
:103D0000E601811105C00E94D52081E08093E60183
:103D1000AE01440F551F4C0F5D1F24E630E0B80183
:103D200080EBDF91CF911F910F910C948821CF935D
:103D3000DF93EC01FB018281882309F43CC1C4308C
:103D4000FDE5DF0760F4CB3F9CE5D90788F49E01D1
:103D500022503C452431310508F02EC109C0C2363D
:103D6000EDE5DE0729F0C63AFDE5DF0709F024C1DD
:103D70000E941A1090938A0280938902C1318CE5C7
:103D8000D80709F4C6C008F042C0C930ECE5DE0728
:103D900009F49BC000F5C5308CE5D80709F485C04F
:103DA00078F4C330ECE5DE0709F478C008F07AC097
:103DB000C230DC4509F0F5C0809189028160EFC016
:103DC000C7309CE5D90709F478C008F07AC0809123
:103DD00089028061E4C0CD30FCE5DF0709F487C0CB
:103DE00058F4CB309CE5D90709F479C008F07BC0C2
:103DF0008091890288606FC0CF30FCE5DF0709F44D
:103E000080C008F082C080918902877FC8C0CE3F01
:103E10009CE5D90709F471C000F5C531FCE5DF0761
:103E200009F485C068F4C3319CE5D90709F475C06D
:103E300008F095C00E94CB09809189028F77AFC0AE
:103E4000CC3FFCE5DF07A9F108F054C0CB3FDC45CF
:103E500009F0A7C080918A0240C0C230EDE5DE07BC
:103E600009F489C058F4C1158DE5D80709F45AC082
:103E700008F069C080918A0282602FC0C236EDE5E9
:103E8000DE0709F47CC0C63AFDE5DF0709F481C00E
:103E9000C330DD4509F085C080E06EC080918902A5
:103EA00082607DC08091890216C0809189028860FD
:103EB00076C080918A0282604FC0809189028062C0
:103EC0006EC08091890280646AC00E94CB09809193
:103ED0008902806864C0846062C081603DC0809156
:103EE00089028E7F5CC0809189028D7F58C080914D
:103EF000890216C080918A0218C080918A028D7F43
:103F00002BC0809189028F7E4AC0809189028F7D6B
:103F100046C0809189028F7B42C080918902877F51
:103F20008B7F3DC080918A028D7F8E7F15C08091EE
:103F3000890282FB222720F991E0922790FB82F9E7
:103F400090FB83F92CC080918A02982F90959170F4
:103F50008E7F892B90FB81F980938A0222C00E9478
:103F6000CB098091890287FB222720F991E09227D3
:103F700090FB87F914C081E00E94B11012C08091BB
:103F8000890284FB222720F991E0922790FB84F993
:103F900006C080918902982F909590FB80F98093BC
:103FA00089028091890290918A020E942B100E94BE
:103FB000CB0980E001C081E0DF91CF910895CF93DC
:103FC000DF9386319C4541F5EB010E941E0F982F2F
:103FD0008A812091620030916300882379F09A7A77
:103FE00081E009F480E08093E701911102C069E269
:103FF00001C065E3C9010E943D220AC08091E7012A
:10400000811102C069E201C065E3C9010E943F223B
:104010000E94600F80E001C081E0DF91CF910895A0
:104020000F931F93CF93DF93C42FD22FFC01828174
:104030008823C9F04093EA010E947A229093E90113
:104040008093E80180E28C0F883008F057C0C77079
:1040500081E001C0880FCA95EAF7DF91CF911F91E7
:104060000F910C9437078091EA01481330C080917A
:10407000E8019091E9010E949222883C910538F56F
:1040800010E21D0FCD17B9F080E28C0F883040F49C
:10409000C77081E001C0880FCA95EAF70E943E0709
:1040A000183028F581E09D2F977001C0880F9A95F0
:1040B000EAF70E943707802F0E942E071830F0F48D
:1040C000D77081E001C0880FDA95EAF70AC080E274
:1040D0008C0F883098F4C77081E001C0880FCA95B2
:1040E000EAF7DF91CF911F910F910C943E07802F3B
:1040F000DF91CF911F910F910C942E07DF91CF91FB
:104100001F910F9108950F939C01CB01243F4CE523
:10411000340731F188F4293DFCE53F07D9F02A3D09
:104120004CE5340779F1283D3C45A9F506E221EE3E
:1041300041EE68ED7CE52BC0263FFCE53F07E1F052
:10414000A8F0273F3C4539F507E225EE46EE67EF3C
:104150007CE51DC007E225EE45EE69ED7CE517C064
:1041600006E221EE40EE64EF7CE511C007E225EEA9
:1041700044EE65EF7CE50BC006E221EE42EE66EF11
:104180007CE505C008E221E045EE6AED7CE50E9491
:10419000102080E008C0FC018281882319F0109271
:1041A000EA0101C081E00F91089511B887E080B95C
:1041B00085B3836085BB86B7846086BF86B7816020
:1041C00086BF86B7806486BF08959F92AF92BF92E4
:1041D000CF92DF92EF92FF920F931F93CF93DF93D3
:1041E000B82EEB010E947A226C01C431D10558F03F
:1041F000CF3F8FEFD80759F0CE0164E170E00E9405
:10420000F0257B0107C0EE24E394F12C03C025E0E8
:10421000E22EF12C84E8A82E94EA992E16BE96BEC2
:104220000E947A228C0106B607FC08C00E947A22FE
:10423000801B910B8E159F05B0F324C081B1887F40
:10424000883039F081B1887F803119F00FEF1FEF8E
:104250001BC0B3B8A6BE0E947A228C0106B607FC2A
:1042600008C00E947A22801B910B8E159F05B0F327
:1042700009C081B1887F883111F0803439F700E0BE
:1042800010E00DC00EEF1FEFCF3F8FEFD80731F2D8
:10429000C6010E9492228C179D0708F4BFCFC80167
:1042A000DF91CF911F910F91FF90EF90DF90CF9012
:1042B000BF90AF909F9008950F931F93CF93DF937C
:1042C000EB0183B984E886BF0E947A228C0106B68E
:1042D00007FC0EC0CF3F8FEFD807C9F30E947A22A8
:1042E000801B910B8C179D0790F38EEF9FEF0BC0F7
:1042F00021B1287F81E090E0283211F480E090E045
:10430000919581959109DF91CF911F910F9108951A
:10431000CF92DF92EF92FF920F931F93CF93DF9391
:104320006B018A017901B9010E94E520E6010C0DBB
:104330001D1DC017D10759F424E926BFDF91CF9185
:104340001F910F91FF90EF90DF90CF90089597FD10
:10435000F3CFB70189910E945C21EBCF90932301A9
:104360008093220108959093F0018093EF010895C6
:10437000E091EF01F091F001309721F00190F08190
:10438000E02D099480E00895E091EF01F091F001B3
:10439000309721F00280F381E02D09940895209157
:1043A000ED013091EE012817390771F09093EE017D
:1043B0008093ED01E091EF01F091F001309721F051
:1043C0000680F781E02D099408952091EB0130914A
:1043D000EC012817390771F09093EC018093EB0101
:1043E000E091EF01F091F001309721F00084F18528
:1043F000E02D09940895FC01329697E080E09150F9
:1044000029F021912223D9F38F5FF9CF08956623F4
:1044100049F0FC01329608962191621729F0E817BD
:10442000F907D1F780E0089581E008959C01FC012F
:1044300032969FEF80E04191461789F09F3F19F433
:10444000411101C0982F8F5F8630A9F79F3F39F047
:10445000F901E90FF11D97FDFA956283089508951A
:104460009C012A5F3F4FFC014281461301C012822A
:10447000019682179307B9F708950C9416220C94AD
:104480003022029626E0FC0111922A95E9F7089560
:1044900008950C9448220C9449220C9448220C94C0
:1044A00048220C944822CF930E944F220E94AC14C1
:1044B0000E944D22C0E08C2F0E94D613892B29F434
:1044C000CF5FC730C1F780E001C081E0CF91089590
:1044D00008958091F30181110C941D0608950E94A6
:1044E000CB090C9424068BE083BF8BEB8CBF82E05E
:1044F00089BF08952FB7F8948091D1029091D2028C
:10450000A091D302B091D4022FBF08952FB7F89491
:104510006091D1027091D2028091D3029091D40225
:104520002FBF08959C014FB7F8948091D1029091CC
:10453000D202A091D302B091D4024FBF821B930B41
:10454000089578941F920F920FB60F9211248F93B3
:104550009F93AF93BF938091D1029091D202A0918B
:10456000D302B091D4020196A11DB11D8093D10256
:104570009093D202A093D302B093D402BF91AF9193
:104580009F918F910F900FBE0F901F90189560E034
:1045900081E090E00E94CE269CE088E10FB6F8947E
:1045A000A89581BD0FBE91BDFFCF0E947A22909346
:1045B000F2018093F10108950E94B7258B9A80E063
:1045C000815041F0A895E7EBFBE03197F1F700C08F
:1045D0000000F6CF8B98789408950E94DA230E9409
:1045E000B3212FEB84ED91E0215080409040E1F722
:1045F00000C0000008958091FC02882389F0109289
:10460000FC020E947A229093F2018093F101809142
:10461000F3018823D1F11092F3010E946F2211C09F
:104620008091F301811111C08091F1019091F2010B
:104630000E949222069728F081E08093F3010E9465
:1046400069228091F301882301F10E9469220E946E
:104650005322882339F1F89421B3939A822F8C60E6
:1046600081BB92B38CE0982792BB3FE54AEE90E085
:10467000315040409040E1F700C0000092B38927DC
:1046800082BB21BB9398789408950E94C0248091A6
:104690000203882329F08091E00284FD0E949C118E
:1046A0000C94812308958091880208950895909133
:1046B000F901981307C02091F7013091F8012617EE
:1046C0003707A9F08093F9017093F8016093F7011F
:1046D0008093F4017093F6016093F50180911903C2
:1046E00084FF05C063E084EF91E00C94BC2408953E
:1046F000BC0184E00C945723BC0183E00C94572345
:104700000895CF93DF93CAE0D0E08091E00284FF68
:1047100018C080910502909106029817E1F028E0F8
:10472000829FC001112468E0895F9D4F0E94B824D8
:104730008091050290E001968F7099278093050281
:104740000AC00E94C02487EB9BE00197F1F700C0EC
:1047500000002197D1F6DF91CF910895CF93DF9399
:10476000EC01A0910602B0E0CD0101968F7099276F
:1047700020910502281779F093E0AA0FBB1F9A95A4
:10478000E1F7A95FBD4F98E0FE0101900D929A9567
:10479000E1F7809306020E94C0240E94812388E0F2
:1047A000FE01ADEFB1E001900D928A95E1F7DF9146
:1047B000CF91089587E790E00895FC01808180768D
:1047C0008032A1F58181813061F484819581892BCA
:1047D00069F58DEF91E09093FE028093FD0288E0F1
:1047E0000895823041F487E892E09093FE0280932E
:1047F000FD0281E008958A3021F48381809387024D
:1048000015C0893099F4828193818115924081F499
:1048100084819581892B61F481E08093FC018681FC
:1048200097819093FB018093FA0102C080E0089584
:104830008FEF08952091FA013091FB01232B71F045
:104840002091FC01213051F4FC0180818093880289
:104850001092FB011092FA0181E008958FEF089504
:104860000895FC0193819330D9F068F4913081F080
:10487000923009F059C08DE996E09093FE02809342
:10488000FD028BE30895913249F19232B9F14CC0A7
:1048900088ED96E09093FE028093FD0282E10895F8
:1048A0008281813099F050F08230F1F58AEE96E005
:1048B0009093FE028093FD028AE0089584E197E0E0
:1048C0009093FE028093FD0284E0089586EF96E0C7
:1048D0009093FE028093FD028CE1089582818823EB
:1048E00029F0813009F588EC96E002C08FEA96E065
:1048F0009093FE028093FD0289E008958481958162
:10490000009751F0019781F488E197E09093FE02BF
:104910008093FD0282E308958AE497E09093FE027B
:104920008093FD0280E4089580E008951F93CF9363
:10493000DF93162FEA01288124FF05C0398128E87A
:104940002327298302C02AE52883212FFC01CE01D9
:104950000296DC0131913D9321501216DCF3612F58
:104960000E94F9031C5F1883DF91CF911F91089576
:1049700040EE52E00C94962449E153E00C949624C6
:10498000CF93DF936091FF02635067FD93C08091E6
:10499000FB02CCE0D0E0C81BD109CD5FDC4F809199
:1049A000FA02803120F4CE010E94302481C08D3281
:1049B00009F06EC0683009F07BC083EC8093D502AB
:1049C0008AE5809384001092F9028881807621F034
:1049D000CE010E94DD2349C09A811092DE028981B6
:1049E000811106C01092DF022EED32E082E038C065
:1049F000853019F49093000330C08630A1F48B8188
:104A0000813041F0823031F0833021F0813211F079
:104A1000823221F4CE010E94312401C080E090E472
:104A20009093F90222C0883089F0893019F490936C
:104A3000020313C08A3069F08B3079F48BE48093E1
:104A4000E10280931A038093ED0207C022E033E075
:104A500002C02EED32E081E003C02EED32E080E0B6
:104A60003093FE022093FD0209C08F3F39F49881F4
:104A700097FD8E8190E89093F90207C09F81911174
:104A800004C09E81981708F4892F8093830010C07A
:104A90008091F90287FF0CC0CE010E941A248F3F3B
:104AA00021F48EE18093840003C081111092830071
:104AB0001092FF028091840084FF4CC0809183009B
:104AC0008F3F09F447C0C82F893008F0C8E08C1B1D
:104AD000809383009091D50288E889278093D5023E
:104AE000CC2359F18091FD029091FE022091F902B0
:104AF00026FF12C0A5EDB2E02C2FAC01455D52405F
:104B0000FA01EA0FFB1FE4911196EC9311972150E3
:104B100011962111F5CF08C0E6EDF2E0DC012C2F53
:104B20003D9131932150E1F701962FEF2C0F820F29
:104B3000911D9093FE028093FD026C2F86ED92E012
:104B40000E94F903CC5FCC3019F08FEF8093830083
:104B5000C093840084E190B39C7031F48150D9F704
:104B6000109200031092F802DF91CF910895CF9335
:104B7000DF9385B7886085BF8BB780688BBFC0EE39
:104B8000D2E08BE48983A9E1B3E011968C9311976D
:104B9000ECEEF2E081838AE588838C938083DF9159
:104BA000CF910895DB018F939F930E945E26BF9162
:104BB000AF91A29F800D911DA39F900DB29F900D6C
:104BC0001124089587FB082E062687FD819567FD31
:104BD00061950E9471260EF4919507FC81950895C8
:104BE000AA1BBB1B51E107C0AA1FBB1FA617B70713
:104BF00010F0A61BB70B881F991F5A95A9F780952F
:104C00009095BC01CD01089597FB072E16F40094F2
:104C100007D077FD09D00E94F02507FC05D03EF4AF
:104C2000909581959F4F0895709561957F4F089558
:104C3000A1E21A2EAA1BBB1BFD010DC0AA1FBB1FA0
:104C4000EE1FFF1FA217B307E407F50720F0A21B12
:104C5000B30BE40BF50B661F771F881F991F1A947F
:104C600069F760957095809590959B01AC01BD01A9
:104C7000CF010895EE0FFF1F0590F491E02D0994E8
:104C80000E944826332312F48A1B9B0B0C9459264E
:104C9000A29FB001B39FC001A39F700D811D11247D
:104CA000911DB29F700D811D1124911D08950E94C8
:104CB0004826B7FF0895821B930B08950E9448264B
:104CC000A59F900DB49F900DA49F800D911D112460
:104CD0000895B7FF0C945E260E945E26821B930BFC
:104CE0000895991B79E004C0991F961708F0961B48
:104CF000881F7A95C9F780950895FC01415050406E
:104D000030F001900616D1F73197CF01089588272A
:104D100099270895FB01DC0104C08D910190801951
:104D200021F441505040C8F7881B990B0895E19930
:104D3000FECF9FBB8EBBE09A99278DB30895A6E165
:104D4000B0E044E050E00C94DD26A8E1B0E042E0A1
:104D500050E00C94DD26262FE199FECF9FBB8EBB41
:104D6000E09A01970DB2021631F02DBB0FB6F89400
:104D7000E29AE19A0FBE08950396272F0E94AC266F
:104D80000E94AB26252F0E94AC26242F0C94AC2623
:104D90000196272F0E94AC260C94AB26262FE19972
:104DA000FECF9FBB8EBB2DBB0FB6F894E29AE19A63
:104DB0000FBE01960895DC01CB01FC01E199FECF05
:104DC00006C0FFBBEEBBE09A31960DB20D9241508A
:0A4DD0005040B8F70895F894FFCFA3
:104DDA00C800B601010102000C000C0C01191A1BD3
:104DEA001C1D1E1F2021225323AE2380237C2378DF
:104DFA00235623FF5AE200E900EA00B500B600B7DD
:104E0A0000CD008301CC008A019201940121022382
:104E1A000224022502260227022A02B300B4006FE6
:104E2A00007000818283E200E900EA00B500B60062
:104E3A00B700CD008301CC008A01920194012102BE
:104E4A00230224022502260227022A02B300B40002
:104E5A006F00700081828390919293949596973710
:104E6A003635343332076061626364666700010273
:104E7A000202020606060909090909090F0F0F0F9E
:104E8A000F0F1515151819191919191919191919A9
:024E9A002324CF
:00000001FF
